:0200000480007A
:100000006F000005732F2034930F80006308FF03F7
:10001000930F90006304FF03930FB0006300FF038E
:10002000130F000063040F0067000F00732F2034CC
:1000300063540F006F00400093E19153171F0000BD
:1000400023223FFC171F000023200FFC6FF01FFF2F
:100050009300000013010000930100001302000050
:100060009302000013030000930300001304000038
:100070009304000013050000930500001306000020
:100080009306000013070000930700001308000008
:10009000930800001309000093090000130A0000F0
:1000A000930A0000130B0000930B0000130C0000D8
:1000B000930C0000130D0000930D0000130E0000C0
:1000C000930E0000130F0000930F0000732540F102
:1000D0006310050097020000938202017390523072
:1000E000735044749702000093820201739052305F
:1000F00073500018970200009382020273905230EE
:10010000B70200809382F2FF7390023B9302F001EA
:100110007390023A7350403097020000938242017C
:100120007390523073502030735030309301000080
:1001300097020000938242ED739052301305100035
:100140001315F501634C05000F00F00F930110002B
:100150009308D0051305000073000000930200000F
:10016000638A020073905210B7B20000938292101B
:100170007390223073500030970200009382420146
:1001800073901234732540F17300203093012000E6
:10019000B70001FF938000F013E7F0F09303F0F055
:1001A0006314771C93013000B710F00F938000FFA9
:1001B00013E7000FB713F00F938303FF6316771A4B
:1001C00093014000B700FF009380F00F13E7F07039
:1001D000B703FF009383F37F6318771893015000F0
:1001E000B7F00FF09380F00013E7000FB7F30FF0B4
:1001F0009383F30F631A771693016000B70001FF32
:10020000938000F093E0000FB70301FF938303FF97
:10021000639C70149301700013020000B710F00F7C
:10022000938000FF13E7000F13030700130212006F
:1002300093022000E31452FEB713F00F938303FFE1
:10024000631473129301800013020000B700FF00D3
:100250009380F00F13E7F070130000001303070002
:100260001302120093022000E31252FEB703FF00B4
:100270009383F37F631A730E9301900013020000BF
:10028000B7F00FF09380F00013E7000F13000000A9
:100290001300000013030700130212009302200052
:1002A000E31052FEB7F30FF09383F30F631E730A4C
:1002B0009301A00013020000B710F00F938000FF1D
:1002C00013E7000F1302120093022000E31652FE00
:1002D000B713F00F938303FF631877089301B000FF
:1002E00013020000B700FF009380F00F130000001E
:1002F00013E7F0F01302120093022000E31452FE01
:100300009303F0FF631277069301C000130200000D
:10031000B7F00FF09380F00013000000130000000E
:1003200013E7000F1302120093022000E31252FEA3
:10033000B7F30FF09383F30F631877029301D000A4
:100340009360000F9303000F639070029301E0002D
:10035000B700FF009380F00F13E0F07093030000EC
:1003600063147000631030020F00F00F638001000F
:100370009391110093E111009308D00513850100BA
:10038000730000000F00F00F930110009308D005D8
:100390001305000073000000731000C0000000008F
:1003A000000000000000000000000000000000004D
:0C03B00000000000000000000000000041
:1010000000000000000000000000000000000000E0
:1010100000000000000000000000000000000000D0
:1010200000000000000000000000000000000000C0
:1010300000000000000000000000000000000000B0
:081040000000000000000000A8
:040000058000000077
:00000001FF
